:10000000B428A00088200C080D040319AF28A920EB
:1000100084132008800664000D280E288C0A03191A
:100020008D0F0B288006AF2823088C0021088D0037
:1000300001308E008F0164003C20031C2F288E0BA2
:100040001B28FF308F0703181B288C07031C8D0704
:10005000031CAF2832308E0000308F001B286D202B
:1000600008308F006E203C208E0C36288F0B3228F3
:100070006E2003140E08080022088400200884174C
:100080008004841300051F192006FF3E080092001B
:10009000220884000930930003105320920C930B24
:1000A0004D280314532884139F1D62280008200440
:1000B0001F1D20068000841700082004031C200652
:1000C00080006E2800082004031C20061F1920064B
:1000D00080008417200980056E281F171F0D063920
:1000E0008C007C208D008C0A7C201F1F8D281F1304
:1000F0008C000230A4208D2800308A000C08820772
:10010000013475340334153400343C340C34D934A0
:10011000FF3A84178005AF288D01E83E8C008D09D9
:10012000FC30031C96288C07031893288C07640066
:100130008D0F93280C189C288C1CA0280000A02848
:10014000080003108D0C8C0CFF3E0318A1280C082E
:10015000AF288C098D098C0A03198D0A08008313B6
:100160000313831264000800831686010D30850096
:1001700083120610831606108312861083168610CB
:1001800083120611831606118312861183168611B7
:1001900083120612831606128312861283168612A3
:1001A000831206138316061383128613831686138F
:1001B000831205168316051283127F30A5007F3047
:1001C000A6007F30A7007F30A8007F30A9007F30D5
:1001D000AA007F30AB007F30AC000530A2000130B8
:1001E000A00004309F000730A300A1011420031CCD
:1001F0004629FF3C031DF6281420031C4629AD00A8
:100200001420031C4629A4000530A2000230A000DF
:1002100004309F002D0847202408472064002D0843
:10022000003C031D15292408A50064002D08013C8D
:10023000031D1C292408A60064002D08023C031D90
:1002400023292408A70064002D08033C031D2A2944
:100250002408A80064002D08043C031D312924084B
:10026000A90064002D08053C031D38292408AA00B4
:1002700064002D08063C031D3F292408AB006400E0
:100280002D08073C031D46292408AC0025088C00D6
:100290008D01063084000130012026088C008D017C
:1002A000063084000230012027088C008D010630C2
:1002B00084000430012028088C008D010630840061
:1002C0000830012029088C008D0106308400103090
:1002D00001202A088C008D01063084002030012086
:1002E0002B088C008D0106308400403001202C0842
:0E02F0008C008D010630840080300120ED2846
:02400E00F53F7C
:00000001FF
